:020000040800F2
:10000000E8070020D5000008A1140008A11200088C
:1000100000000000000000000000000000000000E0
:10002000000000000000000000000000DF170008D2
:100030000000000000000000E9140008E1170008BB
:100040000501000805010008050100080501000878
:1000500005010008ED010008050100080501000880
:100060000501000805010008050100080501000858
:100070000501000805010008050100080501000848
:100080000501000800000000000000000501000854
:100090000000000005010008050100080501000836
:1000A00000000000ED14000805010008050100082B
:1000B0000501000800000000050100080501000816
:1000C0000348854600F080F80048004739250008BD
:1000D000E80700200C4880F308880C480168090EE6
:1000E0000B4A914205D10B480B4901600B480C4962
:1000F00001600C4880470C480047FEE7FEE7FEE73A
:10010000FEE7FEE7FEE70000E8070020040000002D
:100110001F00000018100240010000000000014014
:100120000000000071180008C100000830B50B463F
:10013000014600202022012409E00D46D5409D42C1
:1001400005D31D469540491B254695404019154647
:10015000521E002DF1DC30BD70B50024254600286C
:1001600001DA01244042002901DA01254942FFF762
:10017000DDFFAC4200D04042002C00D0494270BDAF
:100180000549064A08685043054A80180860400837
:100190007047014908607047340000206D4EC64129
:1001A00039300000D2B201E00270401C491EFBD27F
:1001B00070470022F6E710B513460A460446194672
:1001C000FFF7F0FF204610BD064C0125064E05E066
:1001D000E36807CC2B430C3C98471034B442F7D368
:1001E000FFF772FFB82B0008D82B000810B50120CC
:1001F00000F04EF810BD70B50024014620314A7859
:10020000022A03D004218163012416E002681368E6
:100210000E25AB431360026813685B085B00136034
:100220000122056C1346AB40C56B6B604A7000221F
:100230000A70416B002900D08847204670BD31B557
:1002400000F0E0F8009C0546601C00D0641C00F043
:10025000D9F8401BA042FAD338BD000010B50128E0
:1002600010D1062002F0DAF800280BD00920012175
:10027000C00600F0B7F8002805D00022742103481A
:1002800002F0D6F810BD0122F8E70000A801002016
:1002900010B504494A69024202D04861FFF7DEFF07
:1002A00010BD000000040140F8B5002389E00124DE
:1002B0009C402A46A44622407ED04C68022C01D0A5
:1002C000122C0CD1DC08A40027183C6A5D07ED0E47
:1002D0000F26AE40B4430E69AE4026433E62056829
:1002E0005E000324B4400F79A543BF07BF0FB7409A
:1002F0002F4307604D68012D05D0022D03D0112D2D
:1003000001D0122D0ED18568CF68A543B7402F4389
:10031000876047686546AF430D79ED06ED0F9D4058
:100320003D434560C568A5438C68B4402C43C46018
:100330004C68E40044D5264CA56901263543A561E7
:10034000A4699D0834400094224CAD002F19BC686C
:100350009D072E0F0F25B540AC430925ED06A84299
:1003600001D100250AE01C4DA84201D1012505E07C
:100370001A4DA84201D1022500E00525B5402543CC
:10038000BD60174C25684E689543F60300D51543AC
:10039000256065684E689543B60300D515436560D2
:1003A000A5684E689543F60200D51543A560E5683B
:1003B0004E689543B60200E002E000D51543E560C3
:1003C0005B1C0A681546DA4000D070E7F8BD0000F3
:1003D00000100240000001400004004800080048EE
:1003E000000401400069084000D0012070474269C4
:1003F0004A4042617047002A01D0816170478162A2
:100400007047000001480068704700002C00002081
:1004100070B5040005D025466035687A002802D002
:1004200006E0012070BD00202872204600F0B0FEDA
:10043000242068722068016849084900016020464C
:1004400001F056FB0128EDD0606A002802D020465A
:1004500001F0B5FA206841680922D2029143416057
:100460002068816822229143816020688168082287
:100470001143816020680168012211430160204618
:1004800001F002FB70BD000070B504000FD02168C0
:100490001348086021681348086003CC4160206855
:1004A000083C21688860FFF7ADFF054608E00120A1
:1004B00070BDFFF7A7FF401B272801D9032070BD9F
:1004C0002068C0680028F4D120680269E1688A4287
:1004D00001D0016101E004490160002070BD00000D
:1004E000CCCC000055550000AAAA000000680249C3
:1004F0000160002070470000AAAA000002480168BD
:10050000491C0160704700002C00002010B506480F
:100510000168102211430160002000F007F800F08C
:1005200017F8002010BD00000020024010B504465E
:1005300000F0F0F87D21C900FFF7F8FD00F038FD6C
:1005400000222146501E00F037F8002010BD0000A8
:1005500008B5124881690122114381618169114006
:100560000091C26901040A43C261C06900220840C7
:1005700000901146501F00F01FF800221146901EF7
:1005800000F01AF800221146501E00F015F8044839
:10059000016810221143016008BD000000100240F4
:1005A00000000140C106C90E0120884001490860D1
:1005B0007047000000E100E010B500F073FF10BDCF
:1005C000F8B505464E480E460068C007C00FB04259
:1005D0000AD24B480168490849003143016000686C
:1005E000C007C00FB04270D12878464C800705D5AF
:1005F0006068F0218843A968084360602878C007D4
:1006000053D06868012817D0022818D0032819D0C1
:1006100021688907002958DA61688908890001433F
:100620006160FFF7EFFE69680746012913D00229D0
:100630001DD0032927D034E021688903EAE7216827
:100640008901E7E7616BC903E4E7FFF7DBFEC11B44
:100650002D48814223D860680007800F0128F4D11B
:1006600023E0FFF7CFFEC11B2748814217D86068FF
:100670000007800F0228F4D117E0FFF7C3FEC11B6B
:10068000214881420BD860680007800F0328F4D10D
:100690000BE0FFF7B7FEC11B1B48814201D90320C5
:1006A000F8BD60680007800FF3D115480168C907DD
:1006B000C90FB1420BD901684908490031430160B3
:1006C0000068C007C00FB04201D00120F8BD2878F3
:1006D000400706D56068072109028843E968084396
:1006E000606000F02DF86168084A0906090F515C46
:1006F000C840074908600020FFF718FF0020F8BD38
:100700000020024000100240881300009F2B0008C8
:1007100030000020014800687047000030000020D1
:100720000448054900684968044A4905490F515C75
:10073000C84070473000002000100240AF2B000876
:1007400030B516A30FCB89B06C460FC417A30FCBDF
:100750000FC41A494A680C20144604401848042C57
:1007600005D0184B082C04D00C2C00D1184609B029
:1007700030BD9402240F6D462C5DC96A04AD090793
:10078000090FD203695C920F022A02D0032A00D11A
:100790001846FFF7CBFC6043E9E7000002030405BD
:1007A000060708090A0B0C0D0E0F101001020304B6
:1007B00005060708090A0B0C0D0E0F100010024069
:1007C00000127A00006CDC02FEB504460078F04EA0
:1007D000F04DC00748D068680007800F01281FD07F
:1007E00068680007800F022804D16868C003800F82
:1007F000022815D06168012919D001208004002940
:1008000001D0052917D02968B1432960296881439F
:100810002960606800281BD0FFF7F4FD074613E04D
:100820002868800320D56068002876D01CE02868FE
:1008300030432860EDE7296801432960F7E7FFF7B7
:10084000E1FDC01B642869D828688003F7D50BE058
:10085000FFF7D8FD074604E0FFF7D4FDC01B64286E
:10086000F1D828688003F7D4207880073ED56868DF
:100870000007800F14D068680007800F022804D199
:100880006868C003800F01280AD0E0680028286843
:100890001DD0012108432860FFF7B4FD07460BE097
:1008A000286880070BD5E068012836D107E0FFF7FC
:1008B000A9FDC01B0228C6D828688007F7D528687C
:1008C000F82188432169C900084328600EE04008E8
:1008D00040002860FFF796FD074604E0FFF792FD11
:1008E000C01B0228AFD828688007F7D420780007FB
:1008F00024D5E0690028686A11D0012108436862A4
:10090000FFF780FD074604E0FFF77CFDC01B0228CF
:1009100099D8686A8007F7D510E036E1D1E0400841
:1009200040006862FFF76EFD074604E0FFF76AFDCE
:10093000C01B022887D8686A8007F7D4207804276C
:100940004007002861DA00200190E869C00008D45F
:10095000E969B8060143E961E969014001200091B4
:1009600001908D480168C90511D4016882151143B1
:100970000160FFF747FD009005E0FFF743FD009998
:10098000401A642897D884480068C005F5D5A06847
:1009900001280AD0002801D0052811D0286A400873
:1009A00040002862286AB84302E0286A012108430F
:1009B0002862A068002812D0FFF724FD00900AE00A
:1009C000286A38432862F0E7FFF71CFD0099411AB6
:1009D0007248814275D8286A8007F5D50DE0FFF787
:1009E00011FD009006E0FFF70DFD0099411A6B48DC
:1009F000814266D8286A8007F5D40198002804D07F
:100A0000E969012000078143E9612078C00635D5F6
:100A1000606901280CD0401D686B24D0384368639E
:100A2000686B400840006863FFF7ECFC074622E073
:100A3000686B38436863686B012108436863FFF79C
:100A4000E1FC074604E0FFF7DDFCC01B022838D8B4
:100A5000686B8007F7D5686BF8218843A169C900E6
:100A6000084368630AE0B8436863F4E7FFF7CAFC29
:100A7000C01B022825D8686B8007F7D42078800631
:100A800037D568680007800F032813D0686800070F
:100A9000800F022804D16868C003800F032809D0A2
:100AA000206A0028686B16D030436863FFF7AAFC01
:100AB00006460CE0686BC0031BD5206A012864D190
:100AC00017E05BE0FFF79EFC801B022856D8686B9E
:100AD000C003F7D50DE0B0436863FFF793FC06460B
:100AE00004E0FFF78FFC801B022847D8686BC00327
:100AF000F7D4606A002846D069680907890F02297F
:100B000043D0012636060228286805D0B043286065
:100B1000FFF778FC044633E0B0432860FFF772FC2F
:100B2000074604E0FFF76EFCC01B022826D82868A1
:100B30008001F7D4E86A216B000900010843E862EC
:100B4000A16AE06A084369687B22D20391430843A3
:100B50006860286830432860FFF754FC044604E0CE
:100B6000FFF750FC001B022808D828688001F7D541
:100B700009E0FFF747FC001B022801D90320FEBD56
:100B800028688001F5D40020FEBD0120FEBD0000D4
:100B900000000100001002400070004088130000B7
:100BA00070470000F8B504460068426881684B064B
:100BB00005D4CB0703D0530601D5E16C04E08B07C5
:100BC00005D5130603D5216D20468847F8BDFF23C0
:100BD00061331942FAD09306F8D523464D064033C7
:100BE000002D09DA5D7F032D3CD0256E04263543A8
:100BF0002566C568856800958E060125002E08DAF1
:100C0000266E2E4326668668009606684027BE43F9
:100C10000660C80506D5206E0821084320662068B6
:100C200080680090206E0028D0D020684168E026BF
:100C3000B14341605D77900718D02068416889080A
:100C400089004160A06D0B4D002803D04563A06D65
:100C5000FFF7D1FA606D0028B8D04563606DFFF7EB
:100C6000CAFAF8BDC16880680090F8BD2046FFF759
:100C700097FFF8BD5F160008F8B5040007D00026FE
:100C800025464035A662687F002802D005E0012095
:100C9000F8BD2E77204600F04BF802236B772068D2
:100CA00001684022914301600721E06809028842FF
:100CB00001D9002201E0012212030F273F02B842AE
:100CC00002D0884200D0A662276B002F05D188424F
:100CD00001D9236301E001202063A1686068636992
:100CE00008432169194308430123A1695B021940A4
:100CF0000843E1690843216A0843A16A084321685F
:100D00000860616B606AA36908431B0C0427E168F3
:100D10003B40194308432168104348602068C1697B
:100D20007A029143C1612666012068770020F8BDF0
:100D300000B50068114987B088421DD1104882690A
:100D400081140A438261806908400590F020009078
:100D500002200190002103200390029104910920B8
:100D60006946C006FFF7A0FA002211461920FFF7D6
:100D700023FC1920FFF716FC07B000BD003001402E
:100D80000010024070470000F0B504468C46403425
:100D9000217F0025C768964601290CD001212177C3
:100DA000667F4168012E0CD0CA1FFD3A07D18168C9
:100DB000002904D101E00220F0BD042E01D002255B
:100DC00040E0614600291BD07146002918D0002B55
:100DD00016D0617F042901D00521617700210166C9
:100DE000614681638387C38771460164A380E38082
:100DF000072109028F4205D9144AC264144A04E04B
:100E000001251FE0134AC264134A0265012212033E
:100E10008F4202D8E188022903D301684B689343CB
:100E200002E001684B6813434B6001684A68E023A5
:100E30001A434A6000680168490603D401684022E9
:100E400011430160002020772846F0BDFD14000802
:100E50009115000833150008C5150008F8B50122E2
:100E600011024648FFF7C7FA002201214448FFF764
:100E7000C2FA444C444D2078DE2801D0012028706D
:100E8000A078092806D0082824D0012829D00228D3
:100E900051D059E06179207901F01EFA394A2C329B
:100EA0001060E179A07901F017FA5060207A354995
:100EB00040421072607B5072A07BD072E07B9072D7
:100EC000207C1073607C50732F482C31083001F067
:100ED0008FFC39E02B48A2792179203001F0A8FA63
:100EE00032E0284820212038FFF763F92549CD203A
:100EF000203908706078487080278F700220C87091
:100F00000020487103228A7108220B46C8716C3395
:100F10001E5C002E0BD0022E02D0012E02D004E067
:100F2000885402E006463E438E54521CD2B2401C06
:100F30001028EDDB08E00326A05D002804D001F0B6
:100F400035FA761C202EF7DBA078032805D109207E
:100F500000220221C006FFF74EFA0A4A2023D11AC6
:100F60000A48FFF711FF012211460548FFF743FA2F
:100F700001F036FC064940186860F8BD00040048DE
:100F800000140048880100201C00002054000020AC
:100F900010270000042204490428086902D0904365
:100FA000086170471043FBE700E000E07047000075
:100FB000094910B5401E884201D9012010BD074CD7
:100FC00060610321081F00F06DFA0020A061072076
:100FD0002061002010BD0000FFFFFF0000E000E0E6
:100FE00010B5FFF7E3FF10BD70B502462032137F46
:100FF000012B1BD001231377022454770468656802
:101000007026B5436560046865680E6835436560A1
:101010000468A5688026B543A560006884684968AF
:101020000C43846053770020107770BD022070BDA0
:1010300070B5040005D025462035687F002802D011
:1010400006E0012070BD00202877204600F00AF855
:1010500002206877211D206800F038FC01206877A5
:10106000002070BD08B5006801218907884207D1BA
:101070000448C16901221143C161C0691040009058
:1010800008BD0000001002400222014620314A77CC
:1010900002681368012003431360487700207047FB
:1010A000F8B5054604462035287F012817D00127CA
:1010B0002F7702206877226890687726FF23B04355
:1010C0001B02984390600868502837D00EDC202817
:1010D00057D006DC00284ED0102840D14EE0022028
:1010E000F8BD302850D0402839D13CE060282DD0C0
:1010F000702817D001221203801A0ED090422ED1F0
:10110000CB684A688968206800F022FC2068816802
:10111000012292031143816021E020688168C9089F
:10112000C900F8E7CB684A688968206800F010FCBD
:1011300021688868B0433043886010E0CA68496815
:10114000206800F018FC5021206806E0CA68496851
:10115000206800F021FC6021206800F004FC6F771B
:1011600000202877F8BDCA684968206800F003FCB1
:1011700040212068F1E700212068EEE71021206877
:10118000EBE720212068E8E730212068E5E7000050
:1011900000B500680E4987B0884216D10D48C26973
:1011A000012149040A43C261C06908400590042036
:1011B00000901220019001210320039002910491DC
:1011C00009206946C006FFF76FF807B000BD0000B0
:1011D0000044004000100240FFB506460446603659
:1011E000707A83B00D46202858D1002D0CD0059878
:1011F000002809D00120A1680003814207D120699D
:10120000002804D1E80702D0012007B0F0BD307AF1
:10121000012843D0012030720020E0662120707246
:10122000FFF7F0F801902746403705983882059877
:10123000788218E0788A401E788206980090002212
:1012400080212046019B00F0EBFC002818D10120F2
:10125000A1680003814202D12069002812D02168D0
:10126000287808856D1C788A0028E3D106980090BC
:10127000002240212046019B00F0D2FC002808D02B
:101280000320C2E728882168C005C00D0885AD1C71
:10129000E9E72020707200203072B6E70220B4E740
:1012A000FEE70000F0B5474887B042690121890494
:1012B0000A43426142690A400592426909010A43B0
:1012C000426142690A400592426949110A434261FA
:1012D00040694C1208400590002221463A48FFF729
:1012E0008AF8012211463948FFF785F800220221C9
:1012F0003648FFF780F8092000220221C006FFF7D8
:101300007AF8012202213048FFF775F803210920FD
:101310000122C902C006FFF76EF8009400240125DF
:1013200001950294694628480394FEF7BDFF1127F2
:10133000009569462548019702950394FEF7B4FF8E
:101340000226029469462148009601950394FEF70F
:10135000ABFF1F4801900920009569460295C00621
:10136000FEF7A2FF092002946946C0060096019587
:101370000394FEF799FF0820009016480190092079
:1013800069460296C006FEF78FFF029469460E4832
:10139000019700960394FEF787FF0320C002009098
:1013A00009206946019702950394C006FEF77CFF69
:1013B000002203210520FFF7FFF80520FFF7F2F8D0
:1013C00007B0F0BD001002400004004800140048BF
:1013D000000031100000211010B50D480B490160CC
:1013E00000214160816001614161816107220162E8
:1013F00012024162C260816207220163C2624163DC
:10140000FFF73AFC002800D0FEE710BD0030014095
:101410005400002010B50121124886B089070160F0
:1014200000242F21846041600461611E8461C160D9
:10143000FFF7FEFD002800D0FEE70120000300902A
:1014400069460848FFF72CFE002800D0FEE7049408
:1014500004A904480594FFF7C7FD002800D0FEE763
:1014600006B010BDB800002010B50C480A49016054
:10147000E1214902416000218160C1600161816117
:10148000C1610822016242614162FEF7C1FF00288A
:1014900000D0FEE710BD000000440040F80000202E
:1014A000704700008307FF22DB0E9A408907090E70
:1014B000994000280BDA0007000F08388308084815
:1014C0009B001818C36993430B43C361704783089B
:1014D00004489B001B181868904308431860704725
:1014E00000ED00E000E400E07047000010B50248A5
:1014F000FFF758FB10BD00005400002010B5016834
:10150000C968026C1180016C891C0164014640317C
:10151000CA88521ECA80C988002909D101684A6850
:1015200040239A434A60C18F002901D100F06EF830
:1015300010BD10B501464031CC880368026C012C07
:1015400011D9DB681380026C921C0264CA88921E57
:10155000CA80CA88012A0DD1026853680124240375
:101560002343536006E01C7B531C03641470CA8839
:10157000521ECA80C988002909D101684A686023BF
:101580009A434A60C18F002901D100F03FF810BD95
:1015900010B5816B02680988D160816B891C8163F9
:1015A000C18F491EC187C18F00290AD101684A68CD
:1015B00080239A434A604621095A002901D100F04C
:1015C00025F810BD10B5C38F0268816B022B07D3BD
:1015D0000988D160816B891C8163C18F891E05E0F8
:1015E0004B1C836309781173C18F491EC187C18F5A
:1015F00000290AD101684A6880239A434A6046213B
:10160000095A002901D100F001F810BD70B5044657
:10161000FEF7F8FE0246206841682025A943416094
:101620006421204600F024F8002802D0206E2843D0
:101630002066226E204601214030002A04D04177E6
:101640002046FFF7ADFA70BD427F4177042A20465D
:1016500002D0FFF703FC70BDFFF794FB70BD10B51F
:10166000406A002146221152C187FFF799FA10BD46
:10167000F8B50F460B46154600920321044600229A
:10168000C90200F01BF82026002812D13B46002298
:1016900080212046009500F05CF8002809D1032144
:1016A0003B46002249022046009500F007F800283A
:1016B00003D0206E304320660320F8BDF8B51D46E8
:1016C00017460E4604463DE0032149028E4205D1ED
:1016D000002F03D1017B684601700078681C31D06F
:1016E000002D05D0FEF78EFE0699401AA84229D398
:1016F00020684168E022914341606068C11FFD3964
:101700000CD10121A068C903884202D04911884246
:1017100004D1206801684022914301600120A16A40
:101720004003814207D121680A6882430A60216828
:101730000A6802430A600120403460770020207765
:101740000320F8BD206881683140B942BCD1002037
:10175000F8BDF8B51D4617460E46044633E0681C32
:1017600031D0002D05D0FEF74DFE0699401AA84253
:1017700029D320684168E022914341606068C11F1D
:10178000FD390CD10121A068C903884202D049115A
:10179000884204D120680168402291430160012001
:1017A000A16A4003814207D121680A6882430A6026
:1017B00021680A6802430A600120403460770020F3
:1017C00020770320F8BD206881683046884304D024
:1017D0000020B842C3D10020F8BD0120F9E77047CE
:1017E00010B5FEF78BFEFFF7FBFB084C20680028C6
:1017F0000BD000F0F5FF2168884206D900220221B3
:101800000348FEF7F8FD0020206010BD1400002002
:101810000014004810B592B02820009001200890D4
:101820000024079009946846FEF7CEFF002800D0F8
:10183000FEE707200D9003200E900F9401211094D5
:101840000DA8FEF7BDFE002800D0FEE7FEF762FF00
:101850007D21C900FEF76AFCFFF7AAFB0420FFF711
:1018600099FB00221146501EFEF7A6FE12B010BDD5
:10187000134801680122114301604168114A114077
:1018800041600168104A1140016001680122920420
:101890009143016041683F22120491434160C16A53
:1018A00009090901C162016BFF22D432914301632E
:1018B000416B490849004163002181607047000085
:1018C000001002400CB8FF08FFFFF6FEF0B50268FA
:1018D0001A4B0124A4071A4D984203D0A04201D00C
:1018E000A84203D17026B2434E683243154E164FBC
:1018F00098420AD0A04208D0A84206D0134CA04279
:1019000003D0B04201D0B84204D103242402A24340
:10191000CC6822438024A2434C69224302608A6837
:10192000C2620A688262984203D0B04201D0B842D3
:1019300001D10969016301214161F0BD002C014021
:1019400000040040004401400048014000200040E5
:1019500030B58468FF252D021B021343AC430B43B3
:101960002343836030BD826870239A430A43072172
:101970000A438260704730B5036A046A64086400F1
:1019800004628469F025AC43120122430A24A34374
:101990000B438261036230BD30B5036A1024A34358
:1019A00003628469036A0F252D031203AC432243AB
:1019B000A024A343090119438261016230BD10B51F
:1019C000818CC90707D001684A6801235B049A43E8
:1019D000836A1A434A60818C890707D501684A687F
:1019E00001231B049A43C36A1A434A60818C490746
:1019F00007D501684A6801239B049A43036B1A4385
:101A00004A60818C090707D501684A680123DB0316
:101A10009A43436B1A434A60818CC90607D5026812
:101A2000916801231B039943836B19439160818C57
:101A3000890607D501688A6801235B039A43C36B53
:101A40001A438A60818C490612D503685A680121BD
:101A50000905046C8A4322435A60026C8A4207D10A
:101A60000268516803235B059943436C1943516035
:101A7000818C090607D501684A680123DB04806C64
:101A80009A4302434A6010BDF8B500260446C66674
:101A9000FEF7B8FC05461449206888421DD100684D
:101AA000124F000709D501212B4600224905204687
:101AB000009700F0B5F800280DD1206800684007B5
:101AC0000BD501212B46002289052046009700F006
:101AD000A7F8002801D00320F8BD202060346072F0
:101AE000A07226720020F8BD00380140FFFFFF0100
:101AF000F8B504462369A268E5691A4363691020B2
:101B00002B43002125681A432B680E463E4F3B406D
:101B100013432B6023685A6803252D03AA43E56805
:101B20002A435A60236AA26925681A43AB680B27C7
:101B30003F02BB431343AB60344A2568954210D142
:101B4000334A126B9207920F0ED0012A05D0022A57
:101B500005D0032A09D1022007E0042005E008206F
:101B600003E02C4A954200D100200122E369D20310
:101B7000934224D100280CD002280DD0042813D081
:101B8000082817D001260A0912010807400F104340
:101B90002FE0FEF7C5FD09E061681F4A480880187C
:101BA000FEF7C4FA81B2EEE7FEF7CAFD61684000B5
:101BB0004A08F4E76168012248081204EFE70028A8
:101BC00008D0022809D004280BD0082814D00126F8
:101BD0003046F8BDFEF7A4FD05E061680F4A4808ED
:101BE0000CE0FEF7ADFD61684A088018FEF79EFA2A
:101BF00080B22168C860EBE7616848088018FEF78A
:101C000095FA80B2E860E3E7F369FFEF003801403E
:101C100000100240004400400024F40000127A004A
:101C2000FFB581B017460E4604460A9D1DE0681CAC
:101C30001BD0002D05D0FEF7E5FB0499401AA84201
:101C400013D920680168FF22A13291430160206806
:101C50008168490849008160202060346072A07268
:101C600000202072032005B0F0BD2068C169304615
:101C7000884304D00020B842D9D00020F3E70120E7
:101C8000F9E700000FB410B503A9044B044A029809
:101C900000F018F810BC08BC04B018471D23000859
:101CA0003800002002E008C8121F08C1002AFAD13B
:101CB00070477047002001E001C1121F002AFBD1CC
:101CC00070470000FFB58DB00F460546002606E0C0
:101CD00025280AD0109A0F9990476D1C761C2878F9
:101CE0000028F5D1304611B0F0BD00240121674A2B
:101CF000009400E004436D1C2B780846203B98407C
:101D00001042F7D128782E2815D104200443687892
:101D10006D1C2A280AD101CF6D1C00900BE00099A0
:101D20000A225143303940186D1C00902878014632
:101D300030390929F3D92878692843D006DC0028EE
:101D4000D0D063280BD0642804D13BE073280FD097
:101D500075284CD0109A0F999047761C94E03878EB
:101D6000694608720020487202A80190012003E031
:101D7000386801900020C0433F1D61070CD5002446
:101D800000E0641C00998C420FDA8442F9DB01996F
:101D9000095D0029F5D108E0002400E0641C8442BC
:101DA000FCDB0199095D0029F8D1361907E001989B
:101DB00001990078491C0191109A0F999047641E6F
:101DC000F5D261E00A20019001CF002802DA4042FA
:101DD0002D2102E0210504D52B216A461172012133
:101DE00003E0E10701D02021F7E70C9104E00A208D
:101DF000019001CF00210C910BA90B9108E00199F2
:101E0000FEF794F90A460B993032491E0B910A707D
:101E10000028F4D10B9803A9081A2030019060071C
:101E200001D5009801E0012000900199884203DD6E
:101E300001460198081A00E000200024009006E006
:101E400002A8109A005D0F999047641C761C0C98AC
:101E50008442F5DB04E0109A30200F999047761CFD
:101E60000099481E00900029F5DC08E00B980B99BA
:101E70000078491C0B91109A0F999047761C019994
:101E8000481E01900029F1DC6D1C28E7092801009B
:101E900010B5044CE26023812061618100F076F985
:101EA00010BD0000000000201CB5454C6A4601A989
:101EB000444800F0F4FA002844D168460079BA2872
:101EC0001BD24149095CFF2917D039290BD168463B
:101ED0000078012811D13D4A5078401C5070C0074D
:101EE000C00F6A46107068460078002800D0802431
:101EF0004806400C204300F05DF9324800F0DFFA5C
:101F00006846017932486F2906D03A290ED01D293A
:101F100019D0612917D01EE0694609780029018887
:101F200001D02C4A08E00122920309E069460978B1
:101F30000029018802D0284A114002E00122520300
:101F4000114301801CBD6A461278002A028807D01E
:101F5000224B1A4002802A2906D0362904D00BE0F1
:101F60000123DB021A43F5E76A461278002A028849
:101F700007D01B4B1A400280382906D0642904D0B0
:101F80000BE001239B021A43F5E76A461278002A08
:101F900002880DD0134B1A4002807D2901D07E2982
:101FA000D0D1694609780029018805D00E4AC3E7D7
:101FB00001235B021A43EFE7FF220132C0E7000072
:101FC00080800000A8010020A82A00081C00002032
:101FD00006000020FFBF0000FFDF0000FFF7000049
:101FE000FFFB0000FFFD0000FFFE0000F8B500272A
:101FF0001C4C0780064661892069FEF7F3F9012829
:102000002ED1194D284600F02FFDFF2828D0284654
:1020100000F02AFDFF2823D0284600F025FDFF28E8
:102020001ED00025012202211048FEF7E4F9676165
:1020300000240F2700F048F8052810D0391B8840ED
:102040002843641C85B2102CF4DB002202210748CF
:10205000FEF7D1F9044800F007FD35800020F8BDF7
:102060000520F8BD00000020A86100000014004811
:1020700010B5134800F0F0FB00281FD0114910489C
:1020800000F058F90F4B0022587A002801D10122A4
:10209000D203D87A002801D180200243188800B2E8
:1020A00000F0ACF944069888640E144300B200F0C6
:1020B000A5F94006400C204300F07CF810BD00005C
:1020C00024000020C401002070B50D48418900693A
:1020D000FEF788F900280FD10A4D284600F0C4FC0D
:1020E0000446284600F0C0FCFF2C05D0FF2803D092
:1020F000A04203DD012070BD052070BD002070BD31
:1021000000000020A8610000F8B5064600203070ED
:1021100000F0ECF9012806D1114800F0A5FC323896
:10212000292801D30520F8BD0025012202210D48F0
:10213000FEF761F900240727FFF7C6FF0528F2D054
:10214000391B88402843641CC5B2082CF4DB00F01E
:1021500047FB0549FF30F530486135700020F8BD78
:10216000A8610000001400480000002010B5064CD3
:1021700001222189E068FEF73EF901226189206988
:10218000FEF739F910BD00000000002010B5074C23
:102190000220607003202070FFF7E8FF00206061DC
:1021A000024602210248FEF726F910BD0000002079
:1021B00000140048F8B5204F064601220221384697
:1021C000FEF719F91D4C002565610120A070C8209B
:1021D00000F091F8002261892069FEF70CF92220B5
:1021E00000F089F8012261892069FEF704F9402096
:1021F00000F081F8304600F023F8062814D00022C1
:1022000061892069FEF7F7F8402000F074F8012298
:1022100061892069FEF7EFF8A57000220221384697
:10222000FEF7E9F80020F8BDA5700022022138462B
:10223000FEF7E1F80620F8BD001400480000002079
:1022400010B50446000A00F009F8062805D0E0B2EF
:1022500000F004F8062800D0002010BDF8B50025D5
:102260001C4C06460727791B3046C840C00714D0CF
:10227000002261892069FEF7BEF8222000F03BF8B9
:10228000012261892069FEF7B6F861892069FEF7AD
:10229000A9F8012814D1402015E0002261892069A5
:1022A000FEF7A9F8402000F026F801226189206994
:1022B000FEF7A1F861892069FEF794F8012801D0A2
:1022C0000620F8BD222000F016F86D1C082DCADB90
:1022D0000020F8BD000000200902014308B2704749
:1022E00002687F2A01DD7F2103E07E21C9438A4203
:1022F00000DA0160704700B5014600F071FA41183C
:1023000000F06EFA8842FBD300BD000010B5024910
:102310000860FEF7B9FE10BD1800002013B50A23AF
:10232000012269460248FEF757FF00981CBD0000D5
:10233000F800002070B5054600200860486008726B
:102340004872C872887208730C464873284600F0B9
:1023500083FA002823D02168026889182160616807
:10236000426889186160217A027A89182172617A3B
:10237000427A11436172E17AC27A1143E172A17A21
:10238000827A1143A172217B027B11432173617B0D
:10239000407B01436173284600F068FAD6E7204687
:1023A000FFF79EFF201DFFF79BFF70BD70B5440631
:1023B000C109640EC901102C1AD20E4D285D0028E7
:1023C00016D0002910D0022812D1032C02D0062CDE
:1023D00008D104E007482C3800F07AF802E00648FB
:1023E00000F04DFA012002E0012801D10220285519
:1023F00070BD0000D401002024000020C11C06296B
:1024000009D93E214010C9433F2801DB3F2002E0AB
:10241000884200DC0846C0B270470000102803D292
:102420000249085C012800D000207047D401002038
:1024300010B50C46034600F027F8002801D0012013
:1024400010BD19785868445419789868425418781F
:10245000401C4007400F1870002010BD10B5044606
:10246000082000F087F96060082000F083F9A06080
:10247000204600F02DF810BD41780078814201D14E
:10248000012070470020704741780078401C4007C9
:10249000400F814201D1012070470020704710B5E4
:1024A00043780478A34201D1012010BD4468E35C65
:1024B0000B7081684078085C1070002010BD417876
:1024C0000278914203D0491C4907490F4170704777
:1024D00010B5044600202070607008216068FDF788
:1024E00068FE0821A068FDF764FE10BD70B5104CB1
:1024F00061892069FDF776FF0E4D012804D1284639
:1025000000F0B2FAFF280ED00120A070284600F09B
:10251000ABFA7D210901884206DCFF2804D089102E
:10252000884203DA042070BD032070BD012070BD15
:1025300000000020A86100000EB5FDF7E7FFFFF7DF
:1025400069F9FEF7AFFEFEF747FFFEF78DFFFEF7D6
:1025500061FF774875490160032141607549C16099
:102560008160FDF791FF002800D0FEE700270323DC
:102570003A46714971A00097FFF784FB6C48FDF75C
:10258000B5FF6B487430FFF7C1FE00F00DFA6F48DD
:10259000FFF764FF6E4800F041F90020054609226C
:1025A00000900123D20602216A48FFF771FC6748B8
:1025B00020214038FDF7FDFD644A5D482023203A84
:1025C000D11A1030FEF7E0FB614E634C083E5848CC
:1025D000FDF78CFF3078002801D000F007FA00F0FA
:1025E000FFF87168884205D9FF210022013159485E
:1025F000FDF701FF09200821C006FDF7F3FE0028C2
:10260000E5D00320FFF70AFF544A10700620FFF7B9
:1026100005FF2070117801431AD001A8FFF774FD5F
:102620004F4903280F7016D00028D0D16846007992
:10263000000902904548FFF71FFF00280ED04448CC
:1026400000F0F7F8002814D000200546009027E09D
:10265000FFF79CFDBBE7FFF799FDE7E741490298CB
:102660000978884202D0012000900DE000200090FF
:102670000EE03D4902980978884201D0012500E02A
:1026800000250098002803D034480078002804D1A1
:10269000002D05D02078002802D000F093F902E048
:1026A000324800F0E1F96846007900F0F3F80528B7
:1026B00019D002281DD0032822D0042887D123480E
:1026C00020214038FDF775FD204ACD21403A117098
:1026D0008121274891700088410701D40121D170E0
:1026E000C10716D017E020780028B3D0FFF7C0FC50
:1026F0006DE71A4800780028ACD0FFF7D5FB66E7F5
:10270000164800780028A5D019480088FFF752FD28
:102710005DE701211171800701D40120507109206A
:1027200001220221C006FDF766FE50E7003000409E
:1027300044000020FF0F0000622B000825730A20D0
:102740007625642E25642E25640A0000A801002049
:1027500024000020000400480400002003000020A2
:10276000020000200100002000000020A8610000FD
:1027700006000020F0B50B30C108C900144F002638
:10278000144A0FE003688B420BD38B4205D95C1AC5
:102790004318456830C3083B00E04368136002C03B
:1027A00004E0021D10680028ECD13046002803D157
:1027B0003868002801D00020F0BD064A06481060A5
:1027C000064A121AD208D20044C001203860D7E766
:1027D000400000203C000020EC010020E803002025
:1027E000024800680068406A704700001800002036
:1027F00030B50B46024600F024F8002801D0012035
:1028000030BD11785068090140183ACB3AC01078B1
:10281000401C0007000F1070002030BD10B50446AA
:10282000FF200130FFF7A6FF6060204600F027F888
:1028300010BD41780078814201D10120704700200D
:10284000704741780078401C0007000F814201D199
:10285000012070470020704741780278914201D1F1
:10286000002070474068090140187047417802789D
:10287000914203D0491C0907090F4170704710B5F8
:10288000002101704170FF2140680131FDF791FC8A
:1028900010BD0000F8B5010786070509890FB60FBE
:1028A000002D58D03E4C0329207802D002292DD08B
:1028B00073E0032E02D0002E4BD022E085420ED1D1
:1028C000207900280BD0374FFDF75AFC0F21FDF778
:1028D00043FC0806010C38460843FFF76BFC6078A0
:1028E00085420ED1E07800280BD02E4F3F1DFDF71A
:1028F00047FC0F21FDF730FC0806000C3843FFF7BA
:1029000059FC002E29D0022E2CD046E0032E02D0F6
:10291000022E2CD041E085420BD16846FFF766FBC2
:10292000684600880106490E7F2902D10005000F84
:1029300020706078854230D16846FFF757FB6846C3
:1029400000880106490E7F2927D10005000F60701D
:1029500023E0854201D10520F8BD607885421CD175
:102960000220F8BD6078854217D10320F8BD607859
:10297000854212D101220925D402ED0621462846BE
:10298000FDF739FD0648801DFFF730FB0022214688
:102990002846FDF730FD0420F8BD0020F8BD0000FA
:1029A0000000002001600000054800210161416134
:1029B0008161C16101211030C170817170470000D7
:1029C000C401002010B5084C002261892069FDF780
:1029D00012FDFF202D30FFF78EFC01226189206956
:1029E000FDF709FD10BD00000000002012A0FFF758
:1029F00049F9144D0024295D13A0FFF743F9641C25
:102A0000202CF8DB11A0FFF73DF90024FF25134E21
:102A1000013529463046FDF7EAFC6420FDF70FFC3E
:102A2000641C642CF5DBBFF34F8F0E490C48C86063
:102A3000BFF34F8F00BFFDE7535049204552524F1F
:102A4000520A000088010020256420000A72656295
:102A50006F6F74696E672E2E2E0A00000004004806
:102A60000400FA0500ED00E0F8B50746FFF7B8FEF0
:102A70000C4C009061892069FDF7B4FC054609E023
:102A8000FFF7AEFE0099461A002F03D0BE4201D9CF
:102A9000FF20F8BD61892069FDF7A4FCA842EFD0B2
:102AA0003046F8BD00000020FF351213141517162C
:102AB0001A1C191D1B1833300C0D0E0F111020227B
:102AC0001F23211E24360001020305042628252980
:102AD000273238FF060708090B2D2E2B2F2C7B439E
:102AE0003A31397A78637660616264656D47FF597F
:102AF0005B5C4E565758455354555241FFFF0A6789
:102B00006FFFFFFFFFFFFFFF4C7D4BFF7CFF733E1E
:102B1000743B3C773D797275FFFFFFFF7F51FFFFEC
:102B2000FFFFFFFFFF37FFFFFFFFFFFFFFFFFFFF7D
:102B3000FFFFFFFFFFFFFFFFFFFFFFFFFFFFFFFFA5
:102B4000FFFFFFFFFFFFFFFFFFFFFFFFFFFFFFFF95
:102B5000FFFFFFFFFFFFFFFFFFFFFFFFFFFFFF691B
:102B60006B715553423456432050726F746F636FCC
:102B70006C20426F6172640A4170706C652044651C
:102B8000736B746F70204275732028414442290A88
:102B900064656B754E756B656D20323032320000A6
:102BA00000000000000000010203040607080900FD
:102BB0000000000102030400D82B000800000020E0
:102BC00044000000A41C00081C2C00084400002045
:102BD000A4070000B41C0008000000000000FFFF74
:102BE00000000000000000000000000000000000E5
:102BF00000000000000000000000000000000000D5
:102C0000000000000000000000127A000000000038
:0C2C1000000000000000000000000000B8
:04000005080000C12E
:00000001FF
